:020000040800F2
:1000000050050020D50000085D120008ED10000822
:1000100000000000000000000000000000000000E0
:10002000000000000000000000000000CB120008EB
:100030000000000000000000A5120008CD1200081A
:100040000501000805010008050100080501000878
:100050000501000805010008050100080501000868
:100060000501000805010008050100080501000858
:100070000501000805010008050100080501000848
:100080000501000800000000000000000501000854
:100090000000000005010008050100080501000836
:1000A00000000000A9120008050100080501000871
:1000B0000501000800000000050100080501000816
:1000C0000348854600F09CF800480047A51B00083F
:1000D000500500200C4880F308880C480168090E80
:1000E0000B4A914205D10B480B4901600B480C4962
:1000F00001600C4880470C480047FEE7FEE7FEE73A
:10010000FEE7FEE7FEE700005005002004000000C7
:100110001F00000018100240010000000000014014
:100120000000000045130008C100000830B50B4670
:10013000014600202022012409E00D46D5409D42C1
:1001400005D31D469540491B254695404019154647
:10015000521E002DF1DC30BD10B5202A04DB08460C
:10016000203AD040002110BD0B46D340D04020247F
:10017000A21A91400843194610BDD2B201E00270A4
:10018000401C491EFBD270470022F6E710B513460B
:100190000A4604461946FFF7F0FF204610BDF0B5A9
:1001A0001FB40646002082B005464024019100900D
:1001B0001BE0019922460F463046FFF7CDFF049A17
:1001C000059B801A994110D310461946224600F02B
:1001D00029F8361A8F410197224601200021009FFD
:1001E00000F020F838184D4100902046641E002889
:1001F000DFDC019B00982946324607B0F0BD0000C5
:10020000064C0125064E05E0E36807CC2B430C3C69
:1002100098471034B442F7D3FFF756FFA81C0008E4
:10022000C81C000810B5202A04DB0146203A914082
:10023000002010BD914020239C1A0346E34019433F
:10024000904010BD70B50024014620314A78022A42
:1002500003D004218163012416E0026813680E258F
:10026000AB431360026813685B085B0013600122F4
:10027000056C1346AB40C56B6B604A7000220A7078
:10028000416B002900D08847204670BDF8B5002397
:1002900089E001249C402A46A44622407ED04C6836
:1002A000022C01D0122C0CD1DC08A40027183C6AC7
:1002B0005D07ED0E0F26AE40B4430E69AE402643F7
:1002C0003E6205685E000324B4400F79A543BF0772
:1002D000BF0FB7402F4307604D68012D05D0022D99
:1002E00003D0112D01D0122D0ED18568CF68A54302
:1002F000B7402F43876047686546AF430D79ED06E9
:10030000ED0F9D403D434560C568A5438C68B440F2
:100310002C43C4604C68E40044D5264CA5690126F2
:100320003543A561A4699D0834400094224CAD007A
:100330002F19BC689D072E0F0F25B540AC4309252A
:10034000ED06A84201D100250AE01C4DA84201D1CA
:10035000012505E01A4DA84201D1022500E005253E
:10036000B5402543BD60174C25684E689543F6039C
:1003700000D51543256065684E689543B60300D5E2
:1003800015436560A5684E689543F60200D5154390
:10039000A560E5684E689543B60200E002E000D52E
:1003A0001543E5605B1C0A681546DA4000D070E72B
:1003B000F8BD0000001002400000014000040048A9
:1003C00000080048000401400069084000D00120F6
:1003D0007047002A01D08161704781627047000038
:1003E00001480068704700001000002002480168C2
:1003F000491C0160704700001000002010B506483D
:100400000168102211430160002000F007F800F09D
:1004100017F8002010BD00000020024010B504466F
:1004200000F06EF97D21C900FFF780FE00F0AEFC00
:1004300000222146501E00F02FF8002010BD0000C1
:1004400008B50F488169012211438161816911401A
:100450000091C26901040A43C261C06900220840D8
:1004600000901146501F00F017F800221146901E10
:1004700000F012F800221146501E00F00DF808BDE1
:1004800000100240C106C90E0120884001490860E1
:100490007047000000E100E010B500F0E1FE10BD83
:1004A000F8B5044600683E4DC00352D5E869002601
:1004B000C00007D4E96928040143E961E969014002
:1004C0000126009137480168C90510D401688215DA
:1004D00011430160FFF784FF074604E0FFF780FF48
:1004E000C01B642824D82F480068C005F6D5286AA8
:1004F00003273F02384020D06168394081421CD038
:10050000286A2A6AB843012109040A432A622A6A2E
:100510008A432A622862C0070FD0FFF761FF00906C
:1005200008E0FFF75DFF0099411A1F48814201D999
:100530000320F8BD286A8007F3D5286A6168B843AC
:1005400008432862002E04D0E96901200007814396
:10055000E9612078C00705D0286BA1688008800079
:10056000084328632078800605D5286B102188432E
:10057000E168084328632068800305D5286B802143
:1005800088436169084328632088400505D5286BA6
:10059000402188432169084328630020F8BD0000FA
:1005A000001002400070004088130000F8B50546B6
:1005B0004E480E460068C007C00FB0420AD24B48F2
:1005C000016849084900314301600068C007C00F55
:1005D000B04270D12878464C800705D56068F0217C
:1005E0008843A968084360602878C00753D06868CA
:1005F000012817D0022818D0032819D021688907AC
:10060000002958DA61688908890001436160FFF7B1
:10061000E7FE69680746012913D002291DD0032986
:1006200027D034E021688903EAE721688901E7E7F8
:10063000616BC903E4E7FFF7D3FEC11B2D4881427C
:1006400023D860680007800F0128F4D123E0FFF76A
:10065000C7FEC11B2748814217D860680007800F7A
:100660000228F4D117E0FFF7BBFEC11B21488142ED
:100670000BD860680007800F0328F4D10BE0FFF768
:10068000AFFEC11B1B48814201D90320F8BD606841
:100690000007800FF3D115480168C907C90FB1429F
:1006A0000BD9016849084900314301600068C0075F
:1006B000C00FB04201D00120F8BD2878400706D510
:1006C0006068072109028843E9680843606000F018
:1006D0002DF86168084A0906090F515CC8400749AE
:1006E00008600020FFF79AFE0020F8BD00200240BD
:1006F0000010024088130000901C00081400002025
:1007000001480068704700001400002004480549B3
:1007100000684968044A4905490F515CC840704760
:100720001400002000100240A01C000830B516A3E1
:100730000FCB89B06C460FC417A30FCB0FC41A4957
:100740004A680C20144604401848042C05D0184B65
:10075000082C04D00C2C00D1184609B030BD9402EE
:10076000240F6D462C5DC96A04AD0907090FD20339
:10077000695C920F022A02D0032A00D11846FFF7C3
:10078000D5FC6043E9E700000203040506070809F9
:100790000A0B0C0D0E0F10100102030405060708CA
:1007A000090A0B0C0D0E0F100010024000127A0007
:1007B000006CDC02FEB504460078F04EF04DC00738
:1007C00048D068680007800F01281FD068680007BC
:1007D000800F022804D16868C003800F022815D05A
:1007E0006168012919D001208004002901D0052960
:1007F00017D02968B143296029688143296060685E
:1008000000281BD0FFF7ECFD074613E028688003A3
:1008100020D56068002876D01CE028683043286026
:10082000EDE7296801432960F7E7FFF7D9FDC01B11
:10083000642869D828688003F7D50BE0FFF7D0FD5E
:10084000074604E0FFF7CCFDC01B6428F1D82868F8
:100850008003F7D4207880073ED568680007800FB2
:1008600014D068680007800F022804D16868C003AC
:10087000800F01280AD0E068002828681DD00121D7
:1008800008432860FFF7ACFD07460BE028688007A7
:100890000BD5E068012836D107E0FFF7A1FDC01BAA
:1008A0000228C6D828688007F7D52868F821884329
:1008B0002169C900084328600EE040084000286014
:1008C000FFF78EFD074604E0FFF78AFDC01B0228F4
:1008D000AFD828688007F7D42078000724D5E069CE
:1008E0000028686A11D0012108436862FFF778FD8B
:1008F000074604E0FFF774FDC01B022899D8686A18
:100900008007F7D510E036E1D1E04008400068628A
:10091000FFF766FD074604E0FFF762FDC01B0228F3
:1009200087D8686A8007F7D4207804274007002812
:1009300061DA00200190E869C00008D4E969B806CE
:100940000143E961E96901400120009101908D486E
:100950000168C90511D40168821511430160FFF7D0
:100960003FFD009005E0FFF73BFD0099401A642829
:1009700097D884480068C005F5D5A06801280AD03A
:10098000002801D0052811D0286A400840002862BC
:10099000286AB84302E0286A012108432862A06857
:1009A000002812D0FFF71CFD00900AE0286A3843A7
:1009B0002862F0E7FFF714FD0099411A724881425E
:1009C00075D8286A8007F5D50DE0FFF709FD00907E
:1009D00006E0FFF705FD0099411A6B48814266D891
:1009E000286A8007F5D40198002804D0E96901201D
:1009F00000078143E9612078C00635D56069012888
:100A00000CD0401D686B24D038436863686B400885
:100A100040006863FFF7E4FC074622E0686B384358
:100A20006863686B012108436863FFF7D9FC0746D8
:100A300004E0FFF7D5FCC01B022838D8686B80079C
:100A4000F7D5686BF8218843A169C900084368633A
:100A50000AE0B8436863F4E7FFF7C2FCC01B022852
:100A600025D8686B8007F7D42078800637D568686A
:100A70000007800F032813D068680007800F022842
:100A800004D16868C003800F032809D0206A0028B9
:100A9000686B16D030436863FFF7A2FC06460CE093
:100AA000686BC0031BD5206A012864D117E05BE0A6
:100AB000FFF796FC801B022856D8686BC003F7D559
:100AC0000DE0B0436863FFF78BFC064604E0FFF7D8
:100AD00087FC801B022847D8686BC003F7D4606A84
:100AE000002846D069680907890F022943D00126EA
:100AF00036060228286805D0B0432860FFF770FC4E
:100B0000044633E0B0432860FFF76AFC074604E080
:100B1000FFF766FCC01B022826D828688001F7D49E
:100B2000E86A216B000900010843E862A16AE06AF3
:100B3000084369687B22D2039143084368602868B0
:100B400030432860FFF74CFC044604E0FFF748FC04
:100B5000001B022808D828688001F7D509E0FFF7B4
:100B60003FFC001B022801D90320FEBD286880013C
:100B7000F5D40020FEBD0120FEBD000000000100F4
:100B80000010024000700040881300007047000011
:100B9000F8B504460068426881684B0605D4CB0767
:100BA00003D0530601D5E16C04E08B0705D513068D
:100BB00003D5216D20468847F8BDFF2361331942D4
:100BC000FAD09306F8D523464D064033002D09DAB6
:100BD0005D7F032D3CD0256E042635432566C56810
:100BE000856800958E060125002E08DA266E2E43B4
:100BF00026668668009606684027BE430660C805DC
:100C000006D5206E08210843206620688068009081
:100C1000206E0028D0D020684168E026B1434160B2
:100C20005D77900718D02068416889088900416085
:100C3000A06D0B4D002803D04563A06DFFF702FBAC
:100C4000606D0028B8D04563606DFFF7FBFAF8BD12
:100C5000C16880680090F8BD2046FFF797FFF8BD97
:100C6000B9120008F8B5040007D000262546403523
:100C7000A662687F002802D005E00120F8BD2E772B
:100C8000204600F04BF802236B7720680168402271
:100C9000914301600721E0680902884201D90022DE
:100CA00001E0012212030F273F02B84202D088421E
:100CB00000D0A662276B002F05D1884201D923639B
:100CC00001E001202063A16860686369084321692D
:100CD000194308430123A1695B0219400843E169F4
:100CE0000843216A0843A16A084321680860616BD0
:100CF000606AA36908431B0C0427E1683B40194361
:100D000008432168104348602068C1697A02914312
:100D1000C1612666012068770020F8BD00B5006833
:100D2000114987B088421DD11048826981140A4355
:100D30008261806908400590F020009002200190B7
:100D40000021032003900291049109206946C00606
:100D5000FFF79CFA002211461920FFF79DFB19208E
:100D6000FFF790FB07B000BD0030014000100240CB
:100D7000042204490428086902D09043086170479E
:100D80001043FBE700E000E070470000094910B5A0
:100D9000401E884201D9012010BD074C606103212B
:100DA000081F00F05DFA0020A061072020610020EC
:100DB00010BD0000FFFFFF0000E000E010B5FFF7EE
:100DC000E3FF10BD70B502462032137F012B1BD00C
:100DD0000123137702245477046865687026B543AD
:100DE0006560046865680E68354365600468A568D9
:100DF0008026B543A5600068846849680C43846018
:100E000053770020107770BD022070BD70B50400CC
:100E100005D025462035687F002802D006E0012055
:100E200070BD00202877204600F00AF8022068777D
:100E3000211D206800F0B4FA01206877002070BD01
:100E400008B5006801218907884207D10448C169B3
:100E500001221143C161C0691040009008BD00002B
:100E6000001002400222014620314A7702681368CE
:100E7000012003431360487700207047F8B505460A
:100E800004462035287F012817D001272F7702201C
:100E90006877226890687726FF23B0431B02984347
:100EA00090600868502837D00EDC202857D006DC28
:100EB00000284ED0102840D14EE00220F8BD302846
:100EC00050D0402839D13CE060282DD0702817D070
:100ED00001221203801A0ED090422ED1CB684A68AC
:100EE0008968206800F09EFA2068816801229203D8
:100EF0001143816021E020688168C908C900F8E7D2
:100F0000CB684A688968206800F08CFA2168886894
:100F1000B0433043886010E0CA684968206800F038
:100F200094FA5021206806E0CA684968206800F0F9
:100F30009DFA6021206800F080FA6F770020287702
:100F4000F8BDCA684968206800F07FFA402120682F
:100F5000F1E700212068EEE710212068EBE720216F
:100F60002068E8E730212068E5E770B5040005D087
:100F700025466035687A002802D006E0012070BD61
:100F800000202872204600F027F82420687220688C
:100F90000168490849000160204600F013FB012860
:100FA000EDD0606A002802D0204600F072FA206876
:100FB00041680922D20291434160206881682A2257
:100FC000914381602068016801221143016020463D
:100FD00000F0C4FA70BD000000B500680F4987B08A
:100FE000884218D10E488269012189030A4382612F
:100FF0008069084005900320400200900220019083
:1010000000200290032003900120049009206946EB
:10101000C006FFF73BF907B000BD000000380140F3
:1010200000100240FFB5064604466036707A83B071
:101030000D46202858D1002D0CD00598002809D045
:101040000120A1680003814207D12069002804D152
:10105000E80702D0012007B0F0BD307A012843D064
:10106000012030720020E06621207072FFF7B8F98D
:10107000019027464037059838820598788218E015
:10108000788A401E788206980090002280212046AF
:10109000019B00F02FFB002818D10120A16800035C
:1010A000814202D12069002812D021682878088561
:1010B0006D1C788A0028E3D1069800900022402118
:1010C0002046019B00F016FB002808D00320C2E751
:1010D00028882168C005C00D0885AD1CE9E72020DF
:1010E000707200203072B6E70220B4E7FEE700001D
:1010F000F0B5254887B04269012189050A4342615C
:1011000042690A400592426949110A4342614269B3
:101110000A400592426949000A43426140691B4DF9
:1011200008400590012203212846FFF752F90926BD
:10113000F60600220F213046FFF74BF9144F00222C
:1011400002213846FFF745F90320009011200024C2
:1011500001900294694603942846FFF797F80F2000
:101160000125009002946946019503943046FFF7EB
:101170008DF8022000900294694601950394384648
:10118000FFF784F807B0F0BD0010024000140048DB
:101190000004004810B50D480B4901600021416072
:1011A0008160016141618161072201621202416235
:1011B000C260816207220163C2624163FFF752FD90
:1011C000002800D0FEE710BD003001401C000020C8
:1011D00010B50121124886B08907016000242F2133
:1011E000846041600461611E8461C160FFF70EFE8E
:1011F000002800D0FEE7012000030090694608485F
:10120000FFF73CFE002800D0FEE7049404A9044840
:101210000594FFF7D7FD002800D0FEE706B010BD0B
:101220008000002010B50C480A490160E121490204
:10123000416000218160C16001618161C1610C2256
:10124000016242614162FFF790FE002800D0FEE794
:1012500010BD000000380140C000002070470000B1
:101260008307FF22DB0E9A408907090E9940002868
:101270000BDA0007000F0838830808489B0018188D
:10128000C36993430B43C3617047830804489B00C1
:101290001B181868904308431860704700ED00E081
:1012A00000E400E07047000010B50248FFF770FC52
:1012B00010BD00001C00002010B5406A002146222D
:1012C0001152C187FFF762FC10BD704710B5FFF7E0
:1012D0008DF8FFF773FD10BD30B597B020200125C4
:1012E00000240090089509946846FFF763FA0028E7
:1012F00000D0FEE707200D9003200E900F940121EF
:1013000010940DA8FFF752F9002800D0FEE711A8AD
:1013100011951394FFF7C4F8002800D0FEE7FFF7FB
:10132000EFF97D21C900FEF701FFFFF72FFD042033
:10133000FFF71EFD00221146501EFFF7ADF817B053
:1013400030BD00001348016801221143016041686B
:10135000114A114041600168104A11400160016862
:10136000012292049143016041683F22120491439B
:101370004160C16A09090901C162016BFF22D432CF
:1013800091430163416B4908490041630021816039
:1013900070470000001002400CB8FF08FFFFF6FE87
:1013A000F0B502681A4B0124A4071A4D984203D0E5
:1013B000A04201D0A84203D17026B2434E68324306
:1013C000154E164F98420AD0A04208D0A84206D027
:1013D000134CA04203D0B04201D0B84204D1032440
:1013E0002402A243CC6822438024A2434C692243B6
:1013F00002608A68C2620A688262984203D0B04280
:1014000001D0B84201D10969016301214161F0BDF8
:10141000002C01400004004000440140004801400D
:101420000020004030B58468FF252D021B021343C5
:10143000AC430B432343836030BD826870239A43DF
:101440000A4307210A438260704730B5036A046A81
:101450006408640004628469F025AC4312012243ED
:101460000A24A3430B438261036230BD30B5036A93
:101470001024A34303628469036A0F252D0312031A
:10148000AC432243A024A3430901194382610162B2
:1014900030BD10B5818CC90707D001684A680123A7
:1014A0005B049A43836A1A434A60818C890707D593
:1014B00001684A6801231B049A43C36A1A434A60BD
:1014C000818C490707D501684A6801239B049A4328
:1014D000036B1A434A60818C090707D501684A6883
:1014E0000123DB039A43436B1A434A60818CC9068C
:1014F00007D50268916801231B039943836B194345
:101500009160818C890607D501688A6801235B0395
:101510009A43C36B1A438A60818C490612D50368CB
:101520005A6801210905046C8A4322435A60026CFF
:101530008A4207D10268516803235B059943436CD3
:1015400019435160818C090607D501684A68012357
:10155000DB04806C9A4302434A6010BDF8B5002654
:101560000446C666FEF73CFF0546144920688842DB
:101570001DD10068124F000709D501212B4600221A
:1015800049052046009700F0B5F800280DD12068E5
:10159000006840070BD501212B4600228905204613
:1015A000009700F0A7F8002801D00320F8BD202004
:1015B00060346072A07226720020F8BD00380140CD
:1015C000FFFFFF01F8B504462369A268E5691A43E5
:1015D000636910202B43002125681A432B680E46AF
:1015E0003E4F3B4013432B6023685A6803252D036D
:1015F000AA43E5682A435A60236AA26925681A4308
:10160000AB680B273F02BB431343AB60344A2568EA
:10161000954210D1334A126B9207920F0ED0012AD5
:1016200005D0022A05D0032A09D1022007E00420B0
:1016300005E0082003E02C4A954200D10020012259
:10164000E369D203934224D100280CD002280DD0A4
:10165000042813D0082817D001260A091201080708
:10166000400F10432FE0FFF751F809E061681F4A6F
:1016700048088018FEF75AFD81B2EEE7FFF756F8EA
:10168000616840004A08F4E76168012248081204D2
:10169000EFE7002808D0022809D004280BD008283A
:1016A00014D001263046F8BDFFF730F805E0616838
:1016B0000F4A48080CE0FFF739F861684A088018BB
:1016C000FEF734FD80B22168C860EBE76168480826
:1016D0008018FEF72BFD80B2E860E3E7F369FFEFC7
:1016E0000038014000100240004400400024F40093
:1016F00000127A00FFB581B017460E4604460A9DD7
:101700001DE0681C1BD0002D05D0FEF769FE049972
:10171000401AA84213D920680168FF22A1329143E0
:101720000160206881684908490081602020603498
:101730006072A07200202072032005B0F0BD206806
:10174000C1693046884304D00020B842D9D0002077
:10175000F3E70120F9E700000FB410B503A9044B2B
:10176000044A029800F018F810BC08BC04B01847EE
:10177000491B00081800002002E008C8121F08C119
:10178000002AFAD170477047002001E001C1121F02
:10179000002AFBD170470000FFB58FB00F4604460A
:1017A000002606E025280AD0129A11999047641C59
:1017B000761C20780028F5D1304613B0F0BD002506
:1017C0000121A14A009500E00543641C23780846E6
:1017D000203B98401042F7D120782E2815D10420C4
:1017E00005436078641C2A280AD101CF641C00904C
:1017F0000BE000990A22514330394018641C0090D4
:101800002078014630390929F3D920786C280ED088
:1018100004DC4C2813D06A2812D104E074280ED0BE
:101820007A280DD10BE001204005054307E0012196
:10183000090562780D43824201D16D18641C641C55
:101840002078864669284AD008DC0028B4D0582879
:101850006DD0632810D0642808D140E070286BD088
:10186000732812D0752860D0782860D0129A7046FC
:1018700011999047761CE5E0387869460872002097
:10188000487202A80190012003E03868019000200E
:10189000C0433F1D69070CD5002500E06D1C009971
:1018A0008D420FDA8542F9DB0199495D0029F5D1B6
:1018B00008E0002500E06D1C8542FCDB0199495DD4
:1018C0000029F8D1761907E0019801990078491CA0
:1018D0000191129A119990476D1EF5D2B2E00A203B
:1018E000029000216802400F039102280CD001CF22
:1018F000C117844600290DDA62460846524200218B
:10190000814194462D2008E0FF1DFF08FF0003CF12
:101910008446EFE7280504D52B206A461074012081
:101920003CE0E8073AD02020F7E70A2000E010204A
:1019300000210391029007E0102002900021042072
:1019400005430820039100906802400F022810D040
:1019500001CF0021844600200D9028071FD5704636
:1019600070280CD0029A1020039B42401A430CD0DE
:1019700015E0FF1DFF08FF0003CF8446EBE7402082
:101980006A46107401200D900CE06046084306D0B2
:1019900030206A4610747046507402200D907046D4
:1019A000582804D029A001900DA80E900DE02CA07D
:1019B000F9E76046039B029AFEF7F1FB019B844620
:1019C0009B5C0E9A521E0E92137060460843F0D133
:1019D0000E9805A9081A20300190680701D50098D3
:1019E00001E0012000900199884203DD0146019841
:1019F000081A00E000200025009006E004A8129AD2
:101A0000405D119990476D1C761C0D988542F5DB61
:101A100004E0129A302011999047761C0099481ED4
:101A200000900029F5DC08E00E980E990078491C1A
:101A30000E91129A11999047761C0199481E0190B7
:101A40000029F1DC641CB4E609280100303132338E
:101A500034353637383961626364656600000000EA
:101A600030313233343536373839414243444546D4
:101A70000000000010B5044C62602380A06061800B
:101A800000F04AF810BD00000400002070B50D48B9
:101A900041888068FEF798FC00280FD10A4D28463F
:101AA00000F0D4F80446284600F0D0F8611C05D0B8
:101AB000411C03D0A04203DD012070BD052070BD94
:101AC000002070BD0400002010270000F8B50E466D
:101AD000074600F045F8012806D10E4800F0B6F898
:101AE0003238292801D30520F8BD00252C46FFF700
:101AF000CDFF0528F8D0A0402843641CC5B2082CAF
:101B0000F5DB002E02D1034800F0A0F83D70002064
:101B1000F8BD00001027000010B5064C01222188F6
:101B20006068FEF756FC01226188A068FEF751FC50
:101B300010BD00000400002010B502490860FFF746
:101B400091F910BD0000002013B5642301226946FD
:101B50000248FFF767FA00981CBD0000C000002093
:101B600010B50E4841888068FEF72EFC012802D18E
:101B7000002000F06BF80A4800F068F87D210901A8
:101B8000884207DC411C05D04B21C900884203DA9A
:101B9000042010BD032010BD012010BD0400002052
:101BA0001027000008B5FEF729FCFFF795FBFFF7AB
:101BB0009FFAFFF737FBFFF7EDFAFFF709FB16482F
:101BC000FFF7BAFF14482021B030FEF7DDFA1348C2
:101BD000012302460221FFF74DFF11A0FFF7BCFDD4
:101BE0000020694609250870ED0600216846FFF7C8
:101BF0006DFF0446012211462846FEF7EAFB6846BF
:101C0000027821460AA0FFF7A7FD002201212846FD
:101C1000FEF7DFFBE9E70000800000200014004829
:101C200068656C6C6F20776F726C640A000000004E
:101C3000256420307825780A0000000002480068FA
:101C40000068406A7047000000000020F8B50746B1
:101C5000FFF7F4FF0D4C00906188A068FEF7B4FB1D
:101C600005460AE0FFF7EAFF0099461A002F04D064
:101C7000BE4202D90020C043F8BD6188A068FEF7CB
:101C8000A3FBA842EED03046F8BD000004000020BF
:101C9000000000000000000001020304060708091C
:101CA0000000000001020304C81C0008000000201E
:101CB0001C00000078170008E41C00081C0000202D
:101CC0003405000088170008000000000000000034
:101CD00000000000000000000000000000127A0078
:041CE0000000000000
:04000005080000C12E
:00000001FF
